:020000040000FA
:1000000001288316FF3085000830860083128601A0
:1000100095018617AF208613AF208617AF20861371
:10002000AF208617AF208613AF2086176400990A89
:10003000991B1B281E28980A99011628181824288D
:10004000212898182A282728981830282D28181988
:1000500034284128181949285228181959286C2879
:1000600018198928992816288612AF20960A161A78
:100070000617161E061386160616AF20AF20AF20F1
:100080001628861D4128970A17180616171C0612EF
:1000900016288616B9208612B92086190616861DDE
:1000A0000612162806168616B9208612B920B9201F
:1000B0001628960A961D950A961995030616A520E8
:1000C00006128616AF208612A520A520A520A52001
:1000D000A520A520AF201628061605309500A520DE
:1000E000A520A520A520A520A5200612861614303F
:1000F0009500A520A520A520A520A520A520861235
:1001000028309500A520A520A520A520A520A52064
:10011000162886120616861D8928960A961F950AA5
:10012000961B95030612A520970B89288616AF20EB
:1001300016288616A520A520A520A520A520A52047
:10014000A52086120616AF20162815089300143035
:100150009200920BA928930BA72864000800A030F6
:100160009300C8309200920BB328930BB12864001F
:0E017000080014309200920BBB2864000800B7
:00000001FF
